S01A00006275696C642F6D6963613132382F6D61696E2E73726563C2
S11300000C9446000C9463000C9463000C946300FD
S11300100C9463000C9463000C9463000C946300D0
S11300200C9463000C9463000C9463000C946300C0
S11300300C9463000C9463000C9463000C94000112
S11300400C9463000C9463000C9463000C946300A0
S11300500C9463000C9463000C9463000C94630090
S11300600C9463000C9463000C9463000C94630080
S11300700C9463000C9463000C9463000C94630070
S11300800C9463000C9463000C94630011241FBE51
S1130090CFEFD0E1DEBFCDBF11E0A0E0B1E0E0ECF6
S11300A0F2E000E00BBF02C007900D92A030B10750
S11300B0D9F711E0A0E0B1E001C01D92A831B10769
S11300C0E1F70C9494000C940000AC0180E00FB6AE
S11300D007FC81E0F894282F3327E09115018091E3
S11300E015018F5F809315018091150187708093AE
S11300F015019091150180911301981769F022233D
S113010009F07894FF27EE0FFF1FEE5FFE4F408348
S1130110518381E090E00895E0931501222309F0D2
S1130120789480E090E00895CFEFD0E1DEBFCDBFBA
S11301300E94450180E0D99A9598DA9ADA98959ABE
S11301408F5F8739C0F380E0D9989598DA9ADA9866
S1130150959A8F5F8A30C0F3D99ADA9A8AE08093AD
S1130160000110921501109213018FB7F89499278A
S113017010921701DA9AD89AD99A8FBF9FE08FB755
S1130180F894282F332787B78E7F87BF87B78D7F53
S113019087BF80B7886080BF93BF12BE91BF87B707
S11301A0826087BF2FBF78949091130180911501CD
S11301B0981719F480E090E01AC09091130180918F
S11301C013018F5F809313018091130187708093D3
S11301D01301E92FFF27EE0FFF1FEE5FFE4F808113
S11301E0918110821182FC01099581E090E08823BD
S11301F0D9F685B7806285BF889500000000D4CF0A
S113020078941F920F920FB60F9211242F933F935D
S11302108F939F938FB7F894282F332780910101F0
S1130220882369F08091140180931601886080937B
S1130230140183BF8091120181BF109201012FBF6D
S11302408FB7F894382F2091170120FF06C08FB77D
S1130250F8949927DA9A2E7F05C08FB7F8949927D6
S1130260DA982160209317018FBF3FBF9F918F9130
S11302703F912F910F900FBE0F901F9018958FB73D
S1130280F894992708958FBF08951ABA17BA11BA26
S113029082E082B983B9D29AD09AD19A8D9A179A68
S11302A08F9A8E9ABB9A1F9AB89AD79AD39AC09A61
S11302B0DA9AD89AD99A149A1C9A15981D9A08957C
S9030000FC
